:020000040000FA
:100000000000B3200022A0286400F000030EF100DD
:1000100083120B190E288C1A20289A280B11A30B77
:100020001428A1141030A30021189A280608F039CA
:10003000A800290603199A282808A90087219A28C8
:100040008C121A08F2007308FE3A03193828730854
:10005000FD3A03193E287308FC3A03195328730824
:10006000FB3A0319842864007208F300F4019A280B
:1000700064007208BA00FF30F3009A286400F40AA2
:100080007408013A031D47287208B4009A287408BE
:10009000023A031D4E287208B5009A287208B6006D
:1000A000FF30F3009A286400F40A7408013A031D33
:1000B0005C287208B1009A287408023A031D63286C
:1000C0007208B2009A287408033A031D6A2872085D
:1000D000B3009A287408043A031D71287208AF000F
:1000E0009A287408053A031D78287208B0009A28E7
:1000F0007408063A031D7F287208AD009A2872081A
:10010000AE00FF30F3009A286400B7017208F03A9D
:10011000031D93287408B700B8011030B9002115E9
:10012000FF30F3009A2864007208F50074089321E8
:10013000F40A9A286400710E8300F00E700E090014
:1001400000000000640000000000A118AE28211982
:10015000AA28A02821110130D321A028A1103B21D9
:100160003621E020A028AD01AE01AF01B001B10100
:10017000B201B301B401B501B601B701B801B901CB
:1001800039150030BA001030A300A101FF30F30090
:10019000F401640007309F00E0308B008316F830D4
:1001A00085000B3086008530810020308C00CF30F8
:1001B000990024309800831290309800A421080000
:1001C000C230D32134087B212C08303A0319EB28A4
:1001D0002C08CE21ED282030CE2135087B212B089C
:1001E000CE212C08CE213A30CE2136087B212B0897
:1001F000CE212C08CE2108008030D32131087B216C
:100200002C08303A031907292C08CE21092920305F
:10021000CE2132087B212B08CE212C08CE213A306A
:10022000CE2133087B212B08CE212C08CE210800BB
:100230008030D3212F087B212B08CE212C08CE2102
:1002400030087B212B08CE212C08CE2108008030DD
:10025000D3212D087B212B08CE212C08CE212E085E
:100260007B212B08CE212C08CE210800C130D321C0
:100270003A08CE21080052213708031908008030BF
:10028000D3213708F83E0318472937084829083092
:10029000A6003808A70027088C21CE21A70AA60BA4
:1002A0004B2908003708F83E03185829B801080000
:1002B00039087F3903195E29B9030800B91B6A2977
:1002C00008303702380603196729B80A71299030B7
:1002D000B9007129380803196F29B8037129103042
:1002E000B9000800A400FA30A5006400A50B752928
:1002F000A40B73290800AB00AB0E0F39303EAC00E5
:100300002B080F39303EAB002030AA0008006400F3
:100310000C1E87299900080083169B001C141A08DC
:10032000F5008312080083169B0064009C18952931
:100330008B1375089A001C1555309D00AA309D003E
:100340009C148B178312080021148510051132307C
:1003500072213030860005140510053072213030CE
:100360008600051405100130722130308600051416
:100370000510013072212030860005140510831607
:10038000FB30860083120C30D3211C30D32128305F
:10039000D3210130D3210230D32108002114A00041
:1003A000F4210515D7292114A000F4210511EE210F
:1003B00083160B30860083122008F039860005145E
:1003C0000510EE21200EF039860005140510EE21EF
:1003D0008316FB3086008312211008001030A20023
:1003E0006400A20BF0290800051185140514060D00
:1003F00005100514640005100318F629851008007F
:100400004030D3210030CE210030CE210E30CE211D
:100410000E30CE210E30CE210030CE210030CE2144
:100420000030CE210030CE210830CE210C30CE213C
:100430000E30CE210C30CE210830CE210030CE211E
:100440000030CE215830D3210030CE211230CE21C1
:100450001230CE211230CE211230CE211230CE21D8
:0A0460000030CE210030CE2108004C
:02400E00143F5D
:00000001FF
